:100000000C946E000C94D3010C948B000C948B0018
:100010000C948B000C948B000C948B000C948B0034
:100020000C948B000C948B000C948B000C948B0024
:100030000C948B000C948B000C948B000C948B0014
:100040000C948B000C948B000C948B000C948B0004
:100050000C948B000C948B000C948B000C948B00F4
:100060000C948B000C948B0009022200010100A06B
:10007000140904000001030000000921010100012E
:100080002216000705810308006412011001000018
:100090000008C016DF0500010102000114034C0036
:1000A00045004400430074006C00480049004400CF
:1000B00012036F0062006400650076002E0061008C
:1000C0007400040309040600FF0901A101150026BC
:1000D000FF00750895010900B20201C011241FBE7E
:1000E000CFEFD8E0DEBFCDBF11E0A0E0B1E0EAE69F
:1000F000F6E002C005900D92A230B107D9F721E0D9
:10010000A2E0B1E001C01D92AA33B207E1F70E945C
:1001100014030C9433030C940000CF93C62F20914A
:100120000F0124FF19C02091100138E823272093E4
:1001300010012C2FFC01A1E1B1E081918D932150A0
:100140001216DCF36C2F81E191E00E94CF01CC5FAD
:10015000C0930F01CF9108952AE520930F01E9CFB5
:10016000CF93DF9380912001835087FD28C0909129
:100170001C019D3211F5883001F580911D01CCE004
:10018000D0E0C81BD109CC5DDE4F83EC8093040125
:100190008AE580930101109202018881807609F43A
:1001A0005BC0CE010E94F4029F81911104C09E8128
:1001B000981708F4892F80930001109220018091F4
:1001C000010184FF3CC0809100018F3FC1F1C82F25
:1001D000893008F0C8E08C1B8093000180910401F5
:1001E00098E8892780930401CC23E1F040911E0117
:1001F00050911F018091020186FFA6C0A5E0B1E0E9
:10020000FA019C2F84918D9331969150D9F72FEF5D
:100210002C0F30E02F5F3F4F240F351F30931F010D
:1002200020931E016C2F85E091E00E94CF01CC5FEE
:10023000CC3019F08FEF80930001C093010184E16D
:1002400099B1947131F48150D9F710922101109233
:100250001B01DF91CF9108952A8110920D019981A0
:1002600091110AC010920E012DE031E082E030932E
:100270001F0120931E0198CF953029F4209321016E
:100280002DE031E0F4CF963009F047C09B819130EA
:1002900041F48AE890E090931F0180931E0182E16F
:1002A00009C0923059F488E690E090931F01809342
:1002B0001E0182E290E49093020176CF9330C9F45C
:1002C000211108C082EC90E090931F0180931E01E1
:1002D00084E0F0CF213019F480EB90E0DCCF2230C5
:1002E00049F78CE990E090931F0180931E0184E10F
:1002F000E1CF913241F48AE790E090931F0180931F
:100300001E0189E0D7CF9232A9F686EC90E0909357
:100310001F0180931E0186E1CDCF983071F0993096
:1003200019F420932301ACCF9A3059F09B3009F097
:10033000A7CF9BE490931001A3CF23E231E081E0AB
:1003400096CF2DE031E0FBCFDA01E5E0F1E09C2F24
:100350008D9181939150E1F75ACFE9E6F0E08081E9
:1003600082608083E89AEFE0F1E08BE481838AE5A4
:1003700080830895A82FB92F80E090E041E050EAF3
:10038000609530E009C02D9182279795879510F0F0
:1003900084279527305EC8F36F5FA8F30895EADFDE
:1003A0008D939D930895CF93CFB7CF93DF93C3954C
:1003B0004C9BE9F74C9B0BC04C9B09C04C9B07C066
:1003C0004C9B05C04C9B03C04C9B01C08BC06F93E2
:1003D000C0911D01DD27CC5DDE4F2F9365E54C9B61
:1003E00003C02F916F91E6CF0F931F934F9320E09F
:1003F00040E15F9309B1047104FB27F93F9350E09A
:100400003BE039C0147140642F77012F5F5F1EC03D
:10041000406819B114712F7752501FC0406409B160
:100420002F770471D1F15F5F00C023C0406219B122
:100430002F77147191F15F5F00C025C00471102700
:10044000515012F45D5F0000115027952C3F19B1F7
:10045000C8F614710127015027952C3FC8F6422792
:10046000499309B1047110274F73115027952C3F00
:10047000A8F64695469519B1147179F001270150F7
:1004800027952C3F98F66B5A60F3315009B1B0F6BE
:1004900000C011E01CBB002719C03B503195C31BA5
:1004A000D04011E01CBB0881033C09F10B34F9F08A
:1004B00020911B011981110F1213EDCF4A81441FA6
:1004C000093651F10D3211F0013E29F70093220156
:1004D0003F915F914F911F910F912F916F91CCB3ED
:1004E000C0FD65CFDF91CF91CFBFCF9118952091FF
:1004F0002201222369F310912001112391F5343058
:1005000092F13093200120931C0110911D013BE0DA
:10051000311B30931D0127C00091200101300CF5E3
:100520000AE54F7049F43091010134FD1DC000937C
:100530000101C4E0D1E01CC030910F0134FD14C0B2
:1005400000930F01C0E1D1E013C0052710E000C007
:1005500000000BB91AC0052710E0221F1DC010E0D3
:1005600021C04AE502C032ED432FC4E1D0E032E0C1
:100570001AB114615C9A0BB11AB954E120E865E331
:1005800020FF05270BB9279517951C3FF0F66695B8
:10059000B8F7B1F720FF05270BB9279517951C3F32
:1005A000D0F62795179517FF052700001C3F0BB9BC
:1005B000B0F629913A9519F70B7E10912101110F90
:1005C000C651D0400BB911F010931B0111E01CBBB8
:1005D00000611AB11B7E402F4B7E54E05A95F1F713
:1005E0000BB91AB94BB974CFFC0180818076803485
:1005F00049F48181813051F49281892F817090FF7B
:1006000003C0289A80E00895289808958230D1F791
:1006100085B181708093030183E091E090931F0185
:1006200080931E0181E008959EE088E10FB6F89462
:10063000A895809360000FBE909360000E94AD016A
:10064000549A80E0815039F45498209A7894A8956F
:100650000E94B000FCCFA895EFE9FFE03197F1F7D9
:0A06600000C00000EFCFF894FFCFB8
:02066A00FF5A35
:00000001FF
